:1000000000308A008E29000006081E390038031DC2
:1000100038280000000000000000000001309100BE
:10002000111C162883168617831219288316861327
:1000300083120D30850004308C008C0B1D280000CD
:1000400000008316061783120C30850009308C00DF
:100050008C0B2828000000008316061783120D3031
:10006000850004308C008C0B33280000000004282D
:100070000000000000000000000001309100111C91
:100080004528831686178312482883168613831201
:100090000D30850004308C008C0B4C2800000000D3
:1000A0008316061783120C30850009308C008C0BE8
:1000B0005728000000008316061783120D308500B4
:1000C00004308C008C0B622800000000B229003044
:1000D000061801308D000D088F000F088E070F08DD
:1000E0009100111C77288316861783127A288316AD
:1000F000861383120530850004308C008C0B7E281B
:1001000000000000831606138312043085000930B6
:100110008C008C0B892800000000831606178312C0
:100120000530850004308C008C0B94280000000002
:1001300000340030061801308D000D088F000130AA
:100140008E070E089100111CA928831686178312AA
:10015000AC288316861383120D30850004308C0082
:100160008C0BB028000000008316061383120C309D
:10017000850009308C008C0BBB2800000000831622
:10018000061783120D30850004308C008C0BC628B6
:100190000000000000340030061801308D000D080A
:1001A0008F000E088E0701309100111CDB2883168A
:1001B00086178312DE288316861383120D3085007E
:1001C00004308C008C0BE22800000000831606131C
:1001D00083120C30850009308C008C0BED28000058
:1001E00000008316061783120D30850004308C0042
:1001F0008C0BF828000000000034061B2E2900009C
:10020000000000000000000001309100111C0C29CA
:100210008316861783120F298316861383120D30D7
:10022000850004308C008C0B13290000000083161D
:10023000061783120C30850009308C008C0B1E29A8
:10024000000000008316061783120D30850004306D
:100250008C008C0B292900000000FD280000000004
:1002600000000000000001309100111C3B298316A2
:10027000861783123E298316861383120D3085005C
:1002800004308C008C0B42290000000083160617F6
:1002900083120C30850009308C008C0B4D29000036
:1002A00000008316061783120D30850004308C0081
:1002B0008C0B582900000000003400300618013073
:1002C0008D000D088F000E088E079101111C6C29FE
:1002D0008316861783126F298316861383120D30B7
:1002E000850004308C008C0B7329000000008316FD
:1002F000061383120C30850009308C008C0B7E298C
:10030000000000008316061783120D3085000430AC
:100310008C008C0B892900000000003484011F3000
:1003200083058B138B1B912904308C008C1DA02915
:1003300007308101813084000008C0390F38800007
:100340006400813084000008C0390C0480008130D2
:1003500084008013FF3066000030650086010D3098
:10036000850004280030061801308D000D088F002C
:100370000E088E079101111CC1298316861783125E
:10038000C4298316861383120330850004308C0041
:100390008C0BC8290000000083160613831202305C
:1003A000850009308C008C0BD329000000008316D7
:1003B000061783120330850004308C008C0BDE2975
:1003C0000000000067206720672067206720672003
:1003D000672067209920CB20FD205D2167206720C2
:1003E0006720672067206720672067209920CB203F
:1003F000FD205D2167206720672067206720672038
:10040000672067209920CB20FD205D216720672091
:100410006720672067206720672067209920CB200E
:10042000FD20FD20FD20FD20FD20FD20FD20FD20E4
:10043000FD20FD20FD20FD20FD20FD20FD20FD20D4
:10044000FD20FD20FD20FD20FD20FD20FD20FD20C4
:10045000FD20FD20FD20FD20FD20FD20FD20FD20B4
:10046000FD20FD20FD20FD20FD20FD20FD20FD20A4
:10047000FD20FD20FD20FD20FD20FD20FD20FD2094
:10048000FD20FD20FD20FD20FD20FD20FD20FD2084
:0E049000FD20FD20FD20FD20FD20B129630090
:02400E00FA3F77
:00000001FF
